:1000000019C018951895189518951895189518955C
:10001000189518951895189518958FC018951895D6
:100020001895189518951895189518951895189568
:10003000189518958FEF8DBFC8EDE0EC4E2E84E03B
:100040008EBFD4E0F4E05F2EA89584B7082E877F9A
:1000500084BF88E199278093600090936000EEEF61
:10006000F3E0A0E0B1E088278D933197E9F76624AB
:10007000559A5D9A82E0E9E2AAD3A0E0B1E0E5E119
:10008000F1E098E03CD4389A399A3A98BED2409A36
:100090008AE090E0D0D24098419818C05A924A9293
:1000A00087E0D2018C9381E0D5D25A924A9281E0C6
:1000B000D2018C9381E0CED240D1249682E088D2C6
:1000C000409848D182E090E0B6D2409A81EE809389
:1000D0001F015A924A9281E0D2018C9381E0BAD2F8
:1000E00023D1229681E074D287E280931F0180E3BE
:1000F000809320015A924A9282E0D2018C9381E04F
:10010000A9D212D1229681E063D280E08093800050
:1001100085E0809381007894E898E99870916F0069
:10012000716070936F0085E08093810006C073B7A3
:10013000707F716073BF8895FACF0F921F922F92D4
:100140003F924F925F927F92AF92BF920F931F9315
:100150002F933F934F935F936F937F938F939F93CF
:10016000AF93BF93CF93DF93EF93FF938FB78F93AB
:1001700005D274D180EA80931F018AEA809320011E
:100180008BEB809321018CEC8093220180911E01E6
:100190008093230180911D01809324015A924A92F9
:1001A00086E0D2018C9381E055D2BED0229681E0C8
:1001B0000FD282E090E03FD2409A81E090E03BD2C3
:1001C000409884E690E037D280E090E0A2E6B1E08B
:1001D0008D939C93329974C05A924A9287E0D201CF
:1001E0008C9381E037D25A924A9281E0D2018C936B
:1001F00081E030D2A2D0249682E0EAD10091400181
:1002000040E70423A1E6B1E00C93009161010031C5
:1002100009F021C081EE80931F015A924A9281E039
:10022000D2018C9381E016D27FD0229681E0D0D18A
:1002300087E280931F0180E1809320015A924A92C5
:1002400082E0D2018C9381E005D26ED0229681E0CB
:10025000BFD149C035C0003209F013C087E2809396
:100260001F0180E2809320015A924A9282E0D201DB
:100270008C9381E0EFD158D0229681E0A9D133C090
:100280001FC081EE80931F015A924A9281E0D201F1
:100290008C9381E0DFD148D0229681E099D187E22A
:1002A00080931F0180E3809320015A924A9282E05A
:1002B000D2018C9381E0CED137D0229681E088D1D3
:1002C00081E090E0B8D1A2E6B1E086D1A2E6B1E04B
:1002D0000D911C91043650E0150710F009F001C093
:1002E00001C001C077CF5D9881E090E0A4D15D9A14
:1002F0008F918FBFFF91EF91DF91CF91BF91AF9120
:100300009F918F917F916F915F914F913F912F912D
:100310001F910F91BF90AF907F905F904F903F9053
:100320002F901F900F9018954198A881B9819C91AA
:10033000AFE1B1E063D1419A0895419891E0AA817B
:10034000BB815CD1A881B9819C91A0E4B1E04ED180
:10035000419A08958AE280931F0184E380932001EB
:1003600083E48093210180E18093220180E18093E6
:10037000230181E0809324015A924A9286E0D201BF
:100380008C9381E067D1D0DF229681E021D181E298
:1003900080931F0181E0809320015A924A9282E06B
:1003A000D2018C9381E056D1BFDF229681E010D13B
:1003B00082E280931F0181E0809320015A924A9249
:1003C00082E0D2018C9381E045D1AEDF229681E0BC
:1003D000FFD085E280931F0188E2809320015A922A
:1003E0004A9282E0D2018C9381E034D19DDF229643
:1003F00081E0EED081E380931F0185E080932001AE
:100400005A924A9282E0D2018C9381E023D18CDF10
:10041000229681E0DDD086E280931F018FE08093F9
:1004200020015A924A9282E0D2018C9381E012D14B
:100430007BDF229681E0CCD080E280931F018FE0A9
:10044000809320015A924A9282E0D2018C9381E0FB
:1004500001D16ADF229681E0BBD0089580E38093CA
:100460001F0184E38093200183E48093210180E1D4
:100470008093220180E18093230181E08093240115
:100480005A924A9286E0D2018C9381E0E3D04CDF0D
:10049000229681E09DD08AE280931F0184E38093BD
:1004A000200183E48093210180E18093220180E197
:1004B0008093230181E0809324015A924A9286E03E
:1004C000D2018C9381E0C6D02FDF229681E080D0CC
:1004D00081E280931F0181E0809320015A924A9229
:1004E00082E0D2018C9381E0B5D01EDF229681E0BC
:1004F0006FD082E280931F0181E0809320015A92A5
:100500004A9282E0D2018C9381E0A4D00DDF229642
:1005100081E05ED085E280931F0188E28093200114
:100520005A924A9282E0D2018C9381E093D0FCDE11
:10053000229681E04DD086E280931F018FE0809368
:1005400020015A924A9282E0D2018C9381E082D0BB
:10055000EBDE229681E03CD080E280931F018EE0AA
:10056000809320015A924A9282E0D2018C9381E0DA
:1005700071D0DADE229681E02BD0089582E0E9E2A4
:1005800084D05CEC82E0E9E2A2D054E482E0E9E2CB
:100590009ED080E293E04FD082E0E9E2A0E0B1E0BB
:1005A0008BD15EEB82E0E9E292D082E0A8E0B1E09C
:1005B000E9E229E02A93B3D08091080180931D01DC
:1005C0008091090180931E010895481A590A0895DF
:1005D000481A8827580A0895ED91FC91EF5FFF4F64
:1005E000FC93EE9308953197F1F7089515D08C910F
:1005F00015D08D939A95D9F710D008950DD08D917F
:100600000DD09A95E1F709D00895259A24982C9A4F
:10061000239A80E58CBD0895089508958EBD0090BD
:100620004D0007FEFCCF8EB50895689462F80895DA
:10063000E89462F80895EF93FF93EE27E82BE92BF7
:1006400031F0EAEFF0E03197F1F70197D1F7FF9140
:10065000EF910895480E8827581E089591E0882349
:1006600021F08894991F8A95E9F7892F909508952C
:10067000883018F011968850FBCF08950181082B1F
:1006800001831281192312830895D2DFFF27E6DF49
:10069000F5DFEF93FF93E4E7F0E0A5DFFF91EF9143
:1006A000182B128309230183EF93FF93EEE0F0E010
:1006B0009ADFFF91EF911081182309F0B6DFEF93D5
:1006C000FF93E3E6F0E08FDFFF91EF910895C6DF3F
:1006D000FF2721E048E005C0C1DFFF2729915D9198
:1006E00048E0CCDF579510F4182B1283EF93FF935B
:1006F000EAE0F0E078DFFF91EF91182B1283000021
:1007000000000000000000000000000000000000E9
:10071000000000004A9529F72A9509F708959EDF01
:10072000FF27299148E05527A9DF0923018300000D
:1007300000000000000000000000000000000000B9
:10074000000088941081182309F008945795EF93BE
:10075000FF93EAE0F0E047DFFF91EF914A9521F740
:100760005D932A95F9F6089589DF09230183000036
:100770000000000000000000000000000000000079
:100780000000E8941081182309F06894EF93FF9318
:10079000EAE0F0E028DFFF91EF9108956FDF16F4B3
:1007A000182B1283EF93FF93EAE0F0E01CDFFF9138
:1007B000EF91182B128300000000000000000000E1
:1007C0000000000000000000000000000895332732
:1007D000309314013093110158DF0EF458C030915A
:1007E000110130FD54C06627609313016395609337
:1007F000120121E050EF48E074DFB6DF31F9B4DFD9
:1008000032F9632F6670663009F441C0603019F028
:1008100031FB40D025C0609112017091140167171F
:10082000B1F0C0F48F939F93862F8A95A5E1B1E034
:100830001FDF14DF7C9178236894772329F4E894F0
:1008400060911201609313019F918F9109C0689488
:1008500021D006C0E8941ED060911201609313016C
:100860009DDF60911201639560931201613409F07C
:10087000C4CF60911301609314016623E89409F4D6
:10088000689430F930931101E89462F808956894FF
:1008900062F808958F939F93A5E1B1E080911201D2
:1008A0008A95E6DEDBDE7C9116F4782B01C0792395
:1008B0007C939F918F910895AF93BF93EF93FF9394
:1008C00038E0E5E1F1E00D9101933A95E1F7FF9110
:1008D000EF9130E4309314013327309311017CDF22
:1008E00038E0BF91AF91E5E1F1E00D91419104173E
:1008F00019F43A95D1F7089598DE089594E081911E
:080900008D939A95E1F708952B
:00000001FF
